:20000000544A36BDF99932819F271ED601C50A2617C104271CC105276881902707D660C5AC
:2000200002260C39C604D701397F00787EE5908DF34D2A075FBDF9C87EEE207EEEE5BDF920
:20004000C036BDFD83328141270FD6CCC1012630814D262CC606D701398D2C9610847F36F4
:20006000BDEF2D32BDEF2DBDF06A9660852027109610847F36BDEF2D324CBDEF2DBDF06A8D
:2000800039D61326A32096B67D0097104C97118619971E39D660C5202728D61526247F0046
:2000A00052F67802C5042706BDF3B5BDEFB0DE162610CE8800DF16DF1ADF1FDF1CCE8FD033
:2000C000DF1839CEE002DF95CEE2B1DF97CEE2C0DF99CEE489DF9BDF9FCEE6DBDF9D8DB48E
:2000E00039E10EE126E144E150E1FFE28BE10E4D2A09D602C10627167EE59A81042610C665
:2001000001D702D7097F0004D70ADE1ADF1F39CEE0E1D602DFCD58DBCED7CE24037C00CD69
:20012000DECDEE006E00D660C5202705D6101127037F000AC602D702F67D00C47F11270335
:200140007F000939D6111127037F000AC60320E681702604C601207281712604C602206A82
:2001600081732607960926697EE56381742605BDE597205D817226119609270A7F0009967C
:2001800001276A7EE59A7EE0FF8107260EC606D702D601C5082703BDE4B939817D26037E0C
:2001A000E5B980762B1B81052E17CEE1C4DFCD9BCE97CE4F99CD97CDDECDE6007D00092657
:2001C000097EE59A040605070809D708C604D70239966085042616BDE590D613270FCE005D
:2001E00005BDF992CE0002E6B3CA80E7B3C601D703960126058602970139CA04D703398147
:200200000527037EE0F2D608C101275AC1022713960185082650C002D789C608D7017F0060
:200220007A20437F0008D60A262BD6092735D60126157D0013261086029701C601D7037FD6
:20024000000286067EE470BDFB8BBDE59A7F000486157EE470D709D61426EFC602D714C677
:200260004120DA7EE59A7F00087D000A26127D00092715D601C5082707C605D7027EE5B1B4
:20028000BDE59A86047EE4707EE59A81062707811527E67EE59A7F0089BDE5F4D60B5CD1C8
:2002A000612F015FD70B7F0001CE0000BDF99220CFDECF9CD1275FBDF9FACE00037EF990BF
:2002C000BDE2E0DECBA6B385012612CE0002A6B32B0BDECF9CD12705BDF9FA20E37EF99977
:2002E000D601C106260536BDEF2D32D6032713C51026488104260ED601C404D701BDE59A32
:2003000086047EE0EF8103260ECA10D703D667C50127037F0029394D2A04CA20D703C52068
:20032000270AD65C2BF027044D2A0117847FD603C50C26E2C50227107EE3CD7EE40EE353FE
:20034000E387E39AE3ABE35FCEE33ED6047C00047EE114D660C5012706810126662024D6D9
:20036000038102265ECA02D703C5402610965184BFD660C50827028A4097512002D660C56D
:200380000126037F000F39D603C5802609F67D00C47F11262E39D61020F6D66126037C00F3
:2003A00004D603C54027E6D61120E5D603C5402604D6062002D6079705112606D603CA08FB
:2003C000D70339D603CA207F0004D70339D601C1062733D603C5402610D6152F09BDE86F6E
:2003E000D615C50227207EEEE5DE1FB7700001A700089C182602DE169C1C270BDF1F1627EA
:20040000054FC57027E339D603CA20D703399609275BC524263A7D000F26359605D603C5B0
:2004200040270C9707C5082619C601D7142013D6019706C4FD965185402702CA04D701BD4D
:20044000E5CEBDE59ADE1FDF1ABDE8A286062020D603C5042708BDFB8BBDE59A2007C4C1A8
:20046000D703BDE5A0DE1ADF1F861520037EE597D601C106260536BDEF2D328A60CE0006EA
:20048000BDF990CE00027EF99B4D2712BDF79A965EBDF9A416C4E0C160273A7EE4DFC608C7
:2004A000D701D602C10626028D0FCE0000BDF992CE0002BDF9927EF999BDF79AB67D0084BE
:2004C0007FBDF7B2BDF7B28670BDF7B28605BDF7B2BDE5EE39841FBDF7B2BDE5EE20D1D65B
:2004E00060C50127208601BDF7B27F000FB67D00847FBDF7B2BDF7B296612713960B8B3085
:20050000BDF7B2200A96892A06965B970F200E8602BDF7B2D660C50126037F000F96892A4D
:2005200005CEF528201AD665C420D791CEF4E448DFCD9BCE97CE96CD890097CDDECDEE00B9
:20054000AD007EE5D71B0D001F001C010020070000000002601601010000000000000000AF
:20056000000000960A27239709D613270ED660C504261A7F0013BDE8A22006D667C520274C
:2005800009C602D714C641D703397EE59A7EE1FA7F0089C680D77A7F00017F00037F00020D
:2005A0007F000496148102260786019714BDE8A2398640CE00047EE480960927CDD660C5A4
:2005C0008027C7F67802C4EFF778027EE1D1F67802CA10F77802397D007A2A05BDE590207D
:2005E0000A8603BDF7B2960FBDF7B2BDF999CE00077EF99296282609966785102703BDF074
:200600006A3900000000000000000000000000000000000000000000000000000000000037
:200620000000000000000000000000000000000000000000000000000000000000000000BA
:2006400000000000000000000000000000000000000000000000000000000000000000009A
:2006600000000000000000000000000000000000AAD663C504264BD6142647CA80D714973A
:2006800013BDEEAB7F007A96132B10DE23961EB7700001A700BDEFB0BDF02696CC9712CE88
:2006A0000000DFD8B67900841C8A019784B77C00CE0005BDF992CE0000BDF99BCE00027E53
:2006C000F99B7EFB8B8D487D001327013996128103262D8601BDF48B7EF999CE0002BDF9E4
:2006E000927D007A2B15B60001810227028D207D0013270C8601BDF9A420E67EE79B2756FA
:20070000CE0002BDF992CE0000BDF9927EF999BDEE7AF67C00C40AC10227067D007A2B7BA9
:2007200039D6132B76C40F5A271F5A27295A27225A273E5A27655A27105A271A5A27135A77
:2007400027145A27145FD71339860D7C0013B77C0139860A20F54F20F27F00137F007A9691
:2007600014847F97149684849F8A409784B77C00398DE3DE23DFD896D98B5097D996D88950
:200780000097D8DED8099C23270EB7700001A600847F27F1812027EDDFD839DE23B7700081
:2007A00001A60016D11E275F7D007A2B297D00132B1DD5282706D613C510261116847F2785
:2007C0000CC4F0C1902608D667C50827028620B77C019CD827279627814F261496269125D2
:2007E000260E96522732F678028402C4041126287D007A2B037EF047BDF047209E961384AE
:00000001FF
